:020000040000FA
:02000000362A9E
:08000800F100030EF000831665
:1000100003138C1E0F28831203138C1A18288316BF
:1000200003130C1E1728831203130C1A232A312AD8
:1000300083120313F60A1A08F20001307602031D38
:1000400024287208F3001C2A02307602031D2B2894
:100050007208F4001C2A7208F500F6010514F70175
:10006000F31A4928731A5B28F3196D2873197F282E
:10007000F31891287318A328F41BB528741BC728FC
:10008000F41AD928741AEB28F419FD2874190F29C9
:100090002129731AF715731EF711F3197715F31D3C
:1000A00077117319F714731DF710F3187714F31CF5
:1000B000771056223329F319F715F31DF711731929
:1000C0007715731D7711F318F714F31CF7107318D5
:1000D0007714731C771056223A297319F715731D7C
:1000E000F711F3187715F31C77117318F714731CB5
:1000F000F710F41B7714F41F771056224129F318D8
:10010000F715F31CF71173187715731C7711F41B8F
:10011000F714F41FF710741B7714741F771056220E
:1001200048297318F715731CF711F41B7715F41F82
:100130007711741BF714741FF710F41A7714F41E58
:10014000771056224F29F41BF715F41FF711741B73
:100150007715741F7711F41AF714F41EF710741A38
:100160007714741E771056225629741BF715741FC6
:10017000F711F41A7715F41E7711741AF714741E18
:10018000F710F4197714F41D771056225D29F41A2C
:10019000F715F41EF711741A7715741E7711F419F8
:1001A000F714F41DF71074197714741D7710562284
:1001B0006429741AF715741EF711F4197715F41DD4
:1001C00077117419F714741DF710F4187714F41CD0
:1001D000771056226B29F419F715F41DF7117419CD
:1001E0007715741D7711F418F714F41CF7107418B0
:1001F0007714741C7710562272297419F715741D20
:10020000F711F4187715F41C77117418F714741C8F
:10021000F710F51B7714F51F771056227929F4187B
:10022000F715F41CF71174187715741C7711F51B6A
:10023000F714F51FF710751B7714751F77105622EA
:1002400080297418F715741CF711F51B7715F51F25
:100250007711751BF714751FF710F51A7714F51E33
:100260007710562287298510F31A0515F31E0511FC
:10027000851400008510731A0515731E0511851469
:1002800000008510F3190515F31D051185140000F4
:10029000851073190515731D05118514000085104F
:1002A000F3180515F31C051185140000851073184B
:1002B0000515731C0511851400008510F41B051528
:1002C000F41F0511851400008510741B0515741F9B
:1002D0000511851400008510F41A0515F41E05118A
:1002E000851400008510741A0515741E05118514F7
:1002F00000008510F4190515F41D05118514000082
:10030000851074190515741D0511851400008510DC
:10031000F4180515F41C05118514000085107418D7
:100320000515741C0511851400008510F51B0515B5
:10033000F51F0511851400008510751B0515751F27
:100340000511851400008510F51A0515F51E051117
:10035000851400008510751A0515751E0511851484
:1003600000008510F5190515F51D0511851400000F
:10037000851075190515751D05118514000085106A
:10038000F5180515F51C0511851400008510751864
:100390000515751C05118514F91CDE29051185103C
:1003A00005100000000005140000851DD52905106A
:1003B000831603130C16831203131C2A791D132AA8
:1003C000FA010511851000008514000085108519BB
:1003D000FA1785140000851085197A178514000016
:1003E00085108519FA1685140000851085197A166E
:1003F0008514000085108519FA15851400008510F4
:1004000085197A158514000085108519FA1485144C
:100410000000851085197A140510831603130C1635
:10042000831203131C2A051185100510831603136C
:100430000C16831203131C2A83120313981C0F2813
:10044000181218160F28791D272A7A08282A7808E2
:10045000831203139900831603130C1283120313E0
:100460001728700E8300F10E710E0900831203131A
:100470008501860107309F0083160313F83085003D
:10048000FF308600813099002430980083120313D6
:100490009030980085018601F601831603138B17AF
:1004A0000B178C160C1283120313912A0330770258
:1004B000031D5F2A0130F8000130F9000800003008
:1004C0007702031D682A0630F8000130F9000800A1
:1004D00002307702031D712A0330F8000230F90060
:1004E000080001307702031D7A2A0530F800023037
:1004F000F900080077080C390C3C031D842A0230EF
:10050000F8000230F900080077080439043C031DA4
:100510008E2A0430F8000230F90008000430F90097
:040520000800912A14
:02400E00223F4F
:00000001FF
